S02B0000433A2F576F726B2F736F6674776172652F4F70656E424C542F5461726765742F44656D6F2F41524DEF
S3150800400098010020FF410008D9440008D944000857
S31508004010D9440008D9440008D9440008D9440008FE
S31508004020D9440008D9440008D9440008D9440008EE
S31508004030D9440008D9440008D9440008C9440008EE
S31508004040D9440008D9440008D9440008D9440008CE
S31508004050D9440008D9440008D9440008D9440008BE
S31508004060D9440008D9440008D9440008D9440008AE
S31508004070D9440008D9440008D9440008D94400089E
S31508004080D9440008D9440008D9440008D94400088E
S31508004090D9440008D9440008D9440008D94400087E
S315080040A0D9440008D9440008D9440008D94400086E
S315080040B0D9440008D9440008D9440008D94400085E
S315080040C0D9440008D9440008D9440008D94400084E
S315080040D0D9440008D9440008D9440008D94400083E
S315080040E0D9440008D9440008D9440008D94400082E
S315080040F0D9440008D9440008D9440008D94400081E
S31508004100D9440008D9440008D9440008D94400080D
S31508004110D9440008D9440008D9440008D9440008FD
S31508004120D9440008D9440008D9440008D9440008ED
S31508004130D9440008D9440008D9440008D9440008DD
S31508004140D9440008D9440008D9440008D9440008CD
S30908004150EE11AA555F
S315080041542C49072291438D462B482C492C4A00F0BA
S315080041643BF82C482C492D4A00F036F82C482D49A2
S315080041742D4A00F031F82D482D492E4A00F02CF826
S315080041842D482E492E4A00F027F82E482E492F4A44
S3150800419400F022F82E482F49002200F028F82E486D
S315080041A42E49091A082903DB00220260043001603B
S315080041B41F482049884205D00268043003B4904752
S315080041C403BCF7E700208646EC460020002101F0F0
S315080041D44BF8234A9047FEE7884207D0521A05D07F
S315080041E4037801300B700131013AF9D170478842DE
S315080041F402D002700130FAE770471A481A4901607A
S31508004204A6E7000098010020F852000800000020E4
S315080042140C0000207042000870420008D4520008BE
S31508004224F85200080000002000000020D4520008BC
S31508004234D4520008D4520008D4520008D4520008B4
S31508004244D4520008D4520008D4520008F852000880
S315080042540C000020180000201800002098000020F8
S31108004264ED42000808ED00E000400008EC
S3150800427080B500AF01224FF48051024800F0FAFBE6
S3150800428000BF80BD0010014080B582B000AF00F0CD
S3150800429013F97860124B1B687A68D31AB3F5FA7F5C
S315080042A01AD3104B1B78002B09D10E4B01221A701A
S315080042B000224FF480510C4800F0DCFB08E0094B63
S315080042C000221A7001224FF48051074800F0D2FBF1
S315080042D0034A7B68136000E000BF0837BD4680BD0F
S315080042E00C000020100000200010014080B500AF2F
S315080042F000F004F8FFF7C8FFFCE700BF80B500AF81
S3150800430000F00AF800F0ECF800F014F800F0BAF83B
S31508004310FFF7AEFF00BF80BD80B400AF034B044A71
S315080043209A6000BFBD4680BC704700BF00ED00E044
S315080043300040000880B590B000AF0123BB614FF480
S315080043408033FB6100233B620123BB6202237B634C
S315080043504FF48033BB634FF4E013FB6307F1180394
S31508004360184600F09FFB0346002B00D0FEE70F23FC
S315080043707B600223BB600023FB604FF480633B61D4
S3150800438000237B613B1D0221184600F0EFFD034622
S31508004390002B00D0FEE700BF4037BD4680BD00BFFA
S315080043A080B588B000AF354A344B9B6943F00103AA
S315080043B09361324B9B6903F00103FB60FB682F4A4C
S315080043C02E4BDB6943F08053D3612C4BDB6903F03A
S315080043D08053BB60BB68294A284B9B6943F010038E
S315080043E09361264B9B6903F010037B607B6803206F
S315080043F000F086F9002200216FF00B0000F08CF91E
S31508004400002200216FF00A0000F086F90022002140
S315080044106FF0090000F080F9002200216FF0040017
S3150800442000F07AF9002200216FF0030000F074F919
S31508004430002200216FF0010000F06EF90022002131
S315080044404FF0FF3000F068F94FF480533B610123C9
S315080044507B610023BB610223FB6107F11003194648
S31508004460074800F0A9F901224FF48051044800F0EA
S3150800447001FB00BF2037BD4680BD00BF00100240CB
S315080044800010014080B500AF00F0C8FE0246094B97
S31508004490A3FB02239B09184600F05AF9042000F0F2
S315080044A063F9002200214FF0FF3000F035F900BF14
S315080044B080BD00BFD34D621080B500AF00F068F82C
S315080044C00346184680BD00BF80B500AF00F04EF821
S315080044D000F066F900BF80BD80B400AFFEE700BFFC
S315080044E080B500AF084A084B1B6843F010031360F9
S315080044F0032000F005F9002000F008F8FFF750FF48
S315080045000023184680BD00BF0020024080B582B057
S3150800451000AF7860124B1A68124B1B7819464FF495
S315080045207A73B3FBF1F3B2FBF3F3184600F010F914
S315080045300346002B01D001230EE07B680F2B0AD817
S31508004540002279684FF0FF3000F0E6F8064A7B68EB
S315080045501360002300E0012318460837BD4680BDD6
S3150800456008000020040000200000002080B400AFEE
S31508004570054B1B781A46054B1B681344034A136000
S3150800458000BFBD4680BC7047040000201400002010
S3150800459080B400AF024B1B681846BD4680BC704706
S315080045A01400002080B485B000AF78607B6803F003
S315080045B00703FB600C4BDB68BB60BA684FF6FF036A
S315080045C01340BB60FB681A02BB68134343F0BF6322
S315080045D043F40033BB60044ABB68D36000BF14379A
S315080045E0BD4680BC704700BF00ED00E080B400AF58
S315080045F0044BDB6803F4E0631B0A1846BD4680BC1F
S31508004600704700BF00ED00E080B483B000AF0346FA
S315080046103960FB7197F90730002B0BDA0D49FB79E6
S3150800462003F00F03043B3A68D2B21201D2B20B442C
S315080046301A7609E0084997F907303A68D2B21201A2
S31508004640D2B20B4483F8002300BF0C37BD4680BCAA
S31508004650704700BF00ED00E000E100E080B489B0DB
S3150800466000AFF860B9607A60FB6803F00703FB6186
S31508004670FB69C3F10703042B28BF0423BB61FB694D
S315080046800433062B02D9FB69033B00E000237B6158
S315080046900122BB6902FA03F35A1EBB681A407B69FA
S315080046A09A4001217B6901FA03F3591E7B680B4086
S315080046B0134318462437BD4680BC704780B582B080
S315080046C000AF78607B68013BB3F1807F01D301239B
S315080046D00FE00A4A7B68013B53600F214FF0FF3019
S315080046E0FFF792FF054B00229A60044B07221A60D7
S315080046F0002318460837BD4680BD00BF10E000E01D
S3150800470080B582B000AF78607868FFF74BFF00BFCE
S315080047100837BD4680BD00BF80B586B000AF0346EA
S31508004720B9607A60FB7300237B61FFF75FFF7861EE
S315080047307A68B9687869FFF791FF024697F90F30EA
S3150800474011461846FFF760FF00BF1837BD4680BD03
S3150800475080B582B000AF78607868FFF7AFFF034690
S3150800476018460837BD4680BD80B483B000AF786070
S315080047707B68042B06D1094A084B1B6843F00403DF
S31508004780136005E0054A054B1B6823F00403136014
S3150800479000BF0C37BD4680BC704700BF10E000E084
S315080047A080B500AF00F002F800BF80BD80B400AF4E
S315080047B000BFBD4680BC704780B48BB000AF786040
S315080047C039600023FB610023BB6100237B61002362
S315080047D03B6200233B6100237B6227E101227B6A5F
S315080047E002FA03F3FB613B681A68FB691340BB6175
S315080047F0BA69FB699A4240F016813B685B68122BDE
S3150800480034D0122B0DD8022B2BD0022B04D8002B18
S3150800481031D0012B1CD048E0032B43D0112B1BD0E1
S3150800482043E0874A934226D0854A934206D8854A6A
S31508004830934220D0844A93421DD036E0834A93425D
S3150800484019D0834A934216D0824A934213D02CE059
S315080048503B68DB683B6228E03B68DB6804333B6205
S3150800486023E03B68DB6808333B621EE03B68DB6895
S315080048700C333B6219E03B689B68002B02D104238A
S315080048803B6212E03B689B68012B05D108233B621B
S315080048907B68FA691A6108E008233B627B68FA6953
S315080048A05A6102E000233B6200BFBB69FF2B01D8B7
S315080048B07B6801E07B680433FB60BB69FF2B02D889
S315080048C07B6A9B0002E07B6A083B9B003B61FB68B6
S315080048D01A680F213B6901FA03F3DB431A40396A68
S315080048E03B6901FA03F31A43FB681A603B685B6885
S315080048F003F08053002B00F09680574A564B9B696D
S3150800490043F001039361544B9B6903F00103BB60B9
S31508004910BB68524A7B6A9B08023352F823307B6194
S315080049207B6A03F003039B000F2202FA03F3DB43BF
S315080049307A6913407B617B68494A934213D07B6846
S31508004940484A93420DD07B68474A934207D07B6812
S31508004950464A934201D1032306E0042304E00223D6
S3150800496002E0012300E000237A6A02F003029200C3
S3150800497093407A6913437B6138497B6A9B08023303
S315080049807A6941F823203B685B6803F48033002B7F
S3150800499006D03749364B1A68BB6913430B6006E0E5
S315080049A03349334B1A68BB69DB4313400B603B68DA
S315080049B05B6803F40033002B06D02D492C4B5A684C
S315080049C0BB6913434B6006E02949294B5A68BB6902
S315080049D0DB4313404B603B685B6803F48013002B92
S315080049E006D02349224B9A68BB6913438B6006E0BD
S315080049F01F491F4B9A68BB69DB4313408B603B68B2
S31508004A005B6803F40013002B06D01949184BDA68C3
S31508004A10BB691343CB6006E01549154BDA68BB69D9
S31508004A20DB431340CB607B6A01337B627B6A0F2BC7
S31508004A307FF6D4AE00BF2C37BD4680BC704700BF9A
S31508004A4000002110000011100000121000003110A3
S31508004A500000321000002210001002400000014041
S31508004A6000080140000C01400010014000140140FC
S31508004A700004014080B483B000AF78600B467B80A9
S31508004A8013467B707B78002B03D07A887B681A6183
S31508004A9003E07B881A047B681A6100BF0C37BD46A1
S31508004AA080BC704780B586B000AF786000233B6154
S31508004AB07B681B6803F00103002B00F08680924B8D
S31508004AC05B6803F00C03042B0BD08F4B5B6803F079
S31508004AD00C03082B11D18C4B5B6803F48033002B35
S31508004AE00BD0894B1B6803F40033002B6CD07B6812
S31508004AF05B68002B68D101232EE27B685B68B3F5FF
S31508004B00803F06D1804A804B1B6843F4803313608C
S31508004B102EE07B685B68002B0CD17B4A7A4B1B68BE
S31508004B2023F480331360784A774B1B6823F4802379
S31508004B3013601DE07B685B68B3F5A02F0CD1724A41
S31508004B40714B1B6843F4802313606F4A6E4B1B68D6
S31508004B5043F4803313600BE06B4A6B4B1B6823F4FA
S31508004B6080331360684A684B1B6823F480231360FC
S31508004B707B685B68002B13D0FFF70AFD386108E0F5
S31508004B80FFF706FD02463B69D31A642B01D90323B6
S31508004B90E2E15D4B1B6803F40033002BF0D014E010
S31508004BA0FFF7F6FC386108E0FFF7F2FC02463B69BE
S31508004BB0D31A642B01D90323CEE1534B1B6803F4A4
S31508004BC00033002BF0D100E000BF7B681B6803F0C0
S31508004BD00203002B63D04C4B5B6803F00C03002BDD
S31508004BE00BD0494B5B6803F00C03082B1CD1464BD2
S31508004BF05B6803F48033002B16D1434B1B6803F024
S31508004C000203002B05D07B681B69012B01D0012309
S31508004C10A2E13D493C4B1B6823F0F8027B685B69BF
S31508004C20DB0013430B603AE07B681B69002B20D03E
S31508004C30364B01221A60FFF7ABFC386108E0FFF734
S31508004C40A7FC02463B69D31A022B01D9032383E149
S31508004C502D4B1B6803F00203002BF0D02A492A4B80
S31508004C601B6823F0F8027B685B69DB0013430B6063
S31508004C7015E0264B00221A60FFF78AFC386108E027
S31508004C80FFF786FC02463B69D31A022B01D9032398
S31508004C9062E11D4B1B6803F00203002BF0D17B6811
S31508004CA01B6803F00803002B3AD07B689B69002B2E
S31508004CB019D0174B01221A60FFF76AFC386108E021
S31508004CC0FFF766FC02463B69D31A022B01D9032378
S31508004CD042E10D4B5B6A03F00203002BF0D0012082
S31508004CE000F0A6FA1CE00A4B00221A60FFF750FCF7
S31508004CF038610FE0FFF74CFC02463B69D31A022BDA
S31508004D0008D9032328E100BF0010024000004242F0
S31508004D1080044242924B5B6A03F00203002BE9D1FE
S31508004D207B681B6803F00403002B00F0A6800023B1
S31508004D30FB758B4BDB6903F08053002B0DD1884A3A
S31508004D40874BDB6943F08053D361854BDB6903F0FE
S31508004D508053FB60FB680123FB75824B1B6803F4D9
S31508004D608073002B18D17F4A7E4B1B6843F48073EF
S31508004D701360FFF70DFC386108E0FFF709FC0246EF
S31508004D803B69D31A642B01D90323E5E0754B1B68ED
S31508004D9003F48073002BF0D07B68DB68012B06D107
S31508004DA06F4A6F4B1B6A43F0010313622DE07B6861
S31508004DB0DB68002B0CD16A4A694B1B6A23F0010396
S31508004DC01362674A664B1B6A23F0040313621CE0EE
S31508004DD07B68DB68052B0CD1614A614B1B6A43F083
S31508004DE0040313625E4A5E4B1B6A43F001031362B7
S31508004DF00BE05B4A5A4B1B6A23F001031362584ABD
S31508004E00574B1B6A23F0040313627B68DB68002B8D
S31508004E1015D0FFF7BDFB38610AE0FFF7B9FB02467C
S31508004E203B69D31A41F28832934201D9032393E0AE
S31508004E304B4B1B6A03F00203002BEED014E0FFF77E
S31508004E40A7FB38610AE0FFF7A3FB02463B69D31AC2
S31508004E5041F28832934201D903237DE0404B1B6A15
S31508004E6003F00203002BEED1FB7D012B05D13C4A52
S31508004E703B4BDB6923F08053D3617B68DB69002BEE
S31508004E8069D0374B5B6803F00C03082B61D07B684D
S31508004E90DB69022B46D1344B00221A60FFF778FBF8
S31508004EA0386108E0FFF774FB02463B69D31A022B08
S31508004EB001D9032350E02A4B1B6803F00073002B2B
S31508004EC0F0D17B681B6AB3F5803F08D12449244B8F
S31508004ED05B6823F400327B689B6813434B60204869
S31508004EE01F4B5B6823F474127B68196A7B685B6ADC
S31508004EF00B43134343601C4B01221A60FFF748FB20
S31508004F00386108E0FFF744FB02463B69D31A022BD7
S31508004F1001D9032320E0124B1B6803F00073002B12
S31508004F20F0D018E0104B00221A60FFF731FB386109
S31508004F3008E0FFF72DFB02463B69D31A022B01D97D
S31508004F40032309E0064B1B6803F00073002BF0D11E
S31508004F5001E0012300E0002318461837BD4680BD4E
S31508004F6000100240007000406000424280B584B0E4
S31508004F7000AF786039600023FB60724B1B6803F052
S31508004F8007023B689A4210D26E496E4B1B6823F0A3
S31508004F9007023B6813430B606A4B1B6803F0070262
S31508004FA03B689A4201D00123C8E07B681B6803F07E
S31508004FB00203002B08D06449634B5B6823F0F002B8
S31508004FC07B689B6813434B607B681B6803F001038F
S31508004FD0002B6AD07B685B68012B07D15A4B1B688C
S31508004FE003F40033002B15D10123A7E07B685B6827
S31508004FF0022B07D1544B1B6803F00073002B09D111
S3150800500001239BE0504B1B6803F00203002B01D1E0
S31508005010012393E04C494C4B5B6823F003027B6801
S315080050205B6813434B60FFF7B3FAF8607B685B680D
S31508005030012B12D10AE0FFF7ABFA0246FB68D31A36
S3150800504041F28832934201D9032377E03E4B5B68ED
S3150800505003F00C03042BEED127E07B685B68022B78
S315080050601DD10AE0FFF794FA0246FB68D31A41F20B
S315080050708832934201D9032360E0334B5B6803F01F
S315080050800C03082BEED110E0FFF782FA0246FB6804
S31508005090D31A41F28832934201D903234EE02A4BB0
S315080050A05B6803F00C03002BEED1264B1B6803F05C
S315080050B007023B689A4210D92249224B1B6823F003
S315080050C007023B6813430B601E4B1B6803F007027D
S315080050D03B689A4201D0012330E07B681B6803F0E5
S315080050E00403002B08D01849174B5B6823F4E062C9
S315080050F07B68DB6813434B607B681B6803F0080317
S31508005100002B09D01049104B5B6823F460527B686A
S315080051101B69DB0013434B6000F01CF801460A4B81
S315080051205B6803F0F0031B09084AD35C21FA03F312
S31508005130074A13600020FFF7E9F9002318461037DD
S31508005140BD4680BD0020024000100240E85200081B
S315080051500800002090B48AB000AF2B4B3C1D18689D
S3150800516059689A68DB680FC4284A3B4612881A8031
S315080051700023FB610023BB6100237B6200237B6164
S3150800518000233B62224B5B68FB61FB6903F00C035F
S31508005190042B02D0082B03D02DE01E4B3B622DE0DA
S315080051A0FB699B0C03F00F0307F12802134413F85D
S315080051B0243C7B61FB6903F48033002B13D0144B2A
S315080051C05B6803F400335B0C07F12802134413F8F9
S315080051D0283CBB617B690F4A02FB03F2BB69B2FB41
S315080051E0F3F37B6204E07B690B4A02FB03F37B6201
S315080051F07B6A3B6202E0074B3B6200BF3B6A18468C
S315080052002837BD4690BC7047D4520008E4520008BF
S315080052100010024000127A0000093D0080B400AF79
S31508005220024B1B681846BD4680BC70470800002024
S3150800523080B485B000AF78600A4B1B680A4AA2FBA7
S3150800524003235B0A7A6802FB03F3FB6000BFFB6873
S315080052505A1EFA60002BF9D100BF1437BD4680BC30
S31508005260704700BF08000020D34D621080B400AF1D
S31508005270154A154B1B6843F0010313601249124B7C
S315080052805A68124B13404B600F4A0F4B1B6823F0AA
S31508005290847323F4803313600B4A0B4B1B6823F487
S315080052A080231360084A084B5B6823F4FE035360A7
S315080052B0054B4FF41F029A60054B4FF000629A6047
S315080052C000BFBD4680BC7047001002400000FFF8D2
S309080052D000ED00E0FF
S315080052D402030405060708090A0B0C0D0E0F101025
S315080052E4010200000000000000000000010203049F
S309080052F4060708098A
S311080052F8100000000100000000A24A049B
S705080041FFB2
